:020000040000FA
:1000000004EF00F0FFFFFFFF9390060EC16E050E98
:1000100017EC00F0018035EC00F0050E17EC00F055
:10002000019035EC00F007EF00F015EF00F0026EE4
:100030000250036E640E046E0A0E1FEF00F0056E90
:10004000FF0E066E0450086E0350076E770E0624EE
:10005000D8B027EF00F0072E26EF00F0082E24EF8F
:1000600000F0052E22EF00F0120037EF00F00150F3
:10007000816E1200FFFFFFFFFFFFFFFFFFFFFFFF8B
:10008000FFFFFFFFFFFFFFFFFFFFFFFFFFFFFFFF80
:10009000FFFFFFFFFFFFFFFFFFFFFFFFFFFFFFFF70
:1000A000FFFFFFFFFFFFFFFFFFFFFFFFFFFFFFFF60
:1000B000FFFFFFFFFFFFFFFFFFFFFFFFFFFFFFFF50
:0200000400F00A
:020000040030CA
:0E00000000210C0E000180000FC00FE00F4029
:020000040020DA
:08000000FFFFFFFFFFFFFFFF00
:00000001FF
